:1000000012C02CC02BC04FC129C028C027C026C099
:1000100025C024C023C022C021C020C01FC01EC0D4
:100020001DC01CC01BC011241FBECFE5D4E0DEBF25
:10003000CDBF11E0A0E6B0E0E0E9F0E102C005903C
:100040000D92A634B107D9F711E0A6E4B1E001C0E2
:100050001D92AC39B107E1F7F3D518C8D1CF92B3EF
:1000600021B38FE081BB82B3806F82BB9298939A59
:10007000919A00C000C0000080B391980000919A4E
:1000800000009198000087FDF3CF21BB92BB08953B
:10009000DF93CF930F92CDB7DEB78983E0DF9298DD
:1000A0009398919A92B39F7090688981282F2077B6
:1000B000922B92BB000091980000919A92B3829586
:1000C000807F9F70892B82BB000091980F90CF9109
:1000D000DF910895DF93CF930F92CDB7DEB7898379
:1000E000BEDF92989398919A22B38981982F907F3E
:1000F0002F70922B92BB0000919800C000C00000AE
:10010000919A92B38295807F9F70892B82BB000069
:1001100091980F90CF91DF910895DF93CF930F9235
:10012000CDB7DEB789839BDF929A9398919A22B3D9
:100130008981982F907F2F70922B92BB000091980D
:100140000000919A92B38295807F9F70892B82BB29
:10015000000091980F90CF91DF9108950F931F9316
:10016000CF93DF93082F192FC0E0D0E0F8018191E1
:100170008F01D3DF2196C830D105C1F7DF91CF9130
:100180001F910F910895CF93DF9380E081DFC8E046
:10019000D0E080E2C2DF2197E1F780E479DFC8E0B8
:1001A000D0E080E2BADF2197E1F7DF91CF910895A7
:1001B000A898262F372F482F592F71E065B3DA0101
:1001C000C901E5E1B695A79597958795EA95D1F789
:1001D00084709070A070B0706B7F682B65BB220F2D
:1001E000331F441F551F0000A99A0000A9987F5F84
:1001F000793121F7A89AA998AA98089580E090E00B
:10020000FC01EE0FFF1FEA5AFE4F11821082019689
:100210008A309105A9F71092620110926301109241
:1002200064011092650110926601109251011092C2
:1002300050010895209150013091510181E0211524
:10024000310509F480E008958091500190915101A9
:100250000097F9F08091620120E030E001C09A013E
:10026000A9014F5F5F4FFA01EE59FE4F90812E5961
:100270003E4FF90190834930510589F72091500193
:100280003091510121503040309351012093500161
:10029000089580E008958091500190915101009758
:1002A000D1F3D2DF08951F920F920FB60F9211244F
:1002B0002F933F934F935F936F937F938F939F936E
:1002C000AF93BF93CF93DF93EF93FF93369A369913
:1002D000FECF65B1A8EBB0E080E090E045E050E0F3
:1002E0002D91621740F0FC01E354FF4F21E030E014
:1002F0007081671710F020E030E0FC01EE0FFF1F67
:10030000EF01CA5ADE4F0990D881C02DC430D10503
:10031000D9F42223D9F020915001309151012A3093
:100320003105CCF4C0915001D0915101CE59DE4F2E
:10033000888320915001309151012F5F3F4F3093BE
:1003400051012093500107C0222329F4EA5AFE4F9D
:10035000118210820FC0EA5AFE4F208131812F5F37
:100360003F4F31832083208131812530310514F0C6
:100370005183408301968530910509F0B1CFFF91FB
:10038000EF91DF91CF91BF91AF919F918F917F912D
:100390006F915F914F913F912F910F900FBE0F90F2
:1003A0001F901895CF93DF9382E087BB8DEF88BBBA
:1003B0008FEF81BB12BA8FED84BB81E085BB1BBC84
:1003C00086E58ABD8FB58F7B8FBD8EB589608EBD6A
:1003D0008FB588608FBD85E687B983E886B98FB70A
:1003E00080688FBF8FE39DE0A3E081509040A040E4
:1003F000E1F700C0000092989398919A82B38F70B1
:10040000806382BB00C000C000009198A1EEB4E000
:100410001197F1F700C00000919A82B38F7080634A
:1004200082BB00C000C00000919881EE94E001976B
:10043000F1F700C00000919A82B38F70806282BB96
:1004400000C000C000009198A1EEB4E01197F1F750
:1004500000C0000088E23EDE8FE03CDE86E03ADE4F
:1004600081E038DE12BC85B5846085BD14BC8EEF9A
:1004700083BD80E889BFC2DE86DE80E009DE82ECD3
:1004800090E06CDE80E404DE8AEC90E067DE8FE3CF
:1004900092E4AFE081509040A040E1F700C000003E
:1004A0008FB580648FBDA3ECB9E01197F1F700C060
:1004B00000008FB58F7B8FBD66DE80E0E9DD8AE2CC
:1004C00091E04CDE80E4E4DD8CE004DEC8E0D0E0C6
:1004D0008FEF23DE8FE996E8A1E081509040A040A5
:1004E000E1F700C00000219799F78FE0F3DD62E3A8
:1004F00070E080E290E05CDE60E070E080E190E03F
:1005000057DE61E070E080E490E052DE60E070E091
:1005100080E490E04DDEDF91CF91089588E491E092
:1005200060E070E048E050E081D58CE691E068E062
:1005300070E040E350E07AD5089588E491E060E00F
:1005400070E048E050E082D58CE691E068E070E031
:1005500040E350E07BD508952F923F924F925F92F7
:100560006F927F928F929F92AF92BF92CF92DF92C3
:10057000EF92FF920F931F93DF93CF9300D000D0A1
:10058000CDB7DEB7E0914601F0914701309749F4CD
:1005900060915201709153018091540190915501E5
:1005A000E7C0509048014090490130904A012090A6
:1005B0004B0150914C01598360914D016A837091B8
:1005C0004E017B8380914F018C8313E0EE0FFF1F60
:1005D0001A95E1F7E459FE4F80815181F2807381D1
:1005E0000481B581E6809781282F251931E0821793
:1005F00008F030E0452F441981E0541708F080E0FE
:10060000A42FA31B3A2F51E04A1708F050E0852B86
:100610006F2D631951E0F61608F050E0462F481B85
:1006200081E0641708F080E0582B672F621981E0A1
:10063000761708F080E0E62FE51B5E2F71E06E175D
:1006400008F070E0872BA02FF981AF1B71E00A172B
:1006500008F070E06A2F681B81E0A61708F080E0C0
:10066000782BAB2F8A81A81B81E0BA1708F080E0B5
:10067000BA2FB71B7B2FF1E0AB1708F0F0E08F2B00
:10068000FE2DEB81FE1BE1E0EF1608F0E0E0AF2F5E
:10069000A81B8A2FA1E0F81708F0A0E0EA2BBC8184
:1006A0009B1BE0905201F090530100915401109176
:1006B000550137014801990C6608762C43019E1BB1
:1006C00057016801E62CF62C062D162DDED3A0E48A
:1006D000AA2EF2E4BF2EEFE0CE2EDD24EE24FF247E
:1006E00000E010E099D3F901DA01E62E672E022F1F
:1006F000050DFF24F394021708F0FF241F2F140D9B
:10070000552453941F1708F05524EF2DE10FF1E005
:10071000E11708F0F0E05F2A1E2F2A2F230DE1E0F9
:100720002A1708F0E0E0520EF1E0521608F0F0E06F
:10073000EF2B252D3B2F320DF1E03B1708F0F0E0B9
:10074000E30FA1E0E31708F0A0E0FA2B3E2F498168
:100750004E0DE1E04E1508F0E0E0F40FA1E0F417D3
:1007600008F0A0E0EA2B5A81560DE50FC901B80147
:1007700080611EDD61E070E080E490E019DD60E002
:1007800070E080E490E014DD0F900F900F900F90D8
:10079000CF91DF911F910F91FF90EF90DF90CF905D
:1007A000BF90AF909F908F907F906F905F904F9091
:1007B0003F902F900895AF92BF92CF92DF92EF9229
:1007C000FF920F931F93DF93CF93CDB7DEB7289798
:1007D0000FB6F894DEBF0FBECDBF80E289838A8357
:1007E0008B838C838D838E838F8388876091520166
:1007F0007091530180915401909155018E01085FD1
:100800001F4F5E010894A11CB11C3AE0C32ED12CED
:10081000E12CF12CA701960195D3605DF80162935C
:100820008F01B901CA01EA15FB05A1F7E091460164
:10083000F0914701EE0FFF1FE455FF4F808128DC48
:100840008EE26BDC80E024DC6E010894C11CD11CBC
:1008500000E010E0802FE0914601F0914701EE0F9B
:10086000FF1FE455FF4F20813181021713070CF061
:100870008F5F0EDCF60181916F014FDC0F5F1F4F20
:100880000730110539F78091600190916101E09185
:100890004601F0914701EE0FFF1FE455FF4F208105
:1008A0003181821793070CF08F5FF2DB28960FB629
:1008B000F894DEBF0FBECDBFCF91DF911F910F9196
:1008C000FF90EF90DF90CF90BF90AF9008951F936F
:1008D00072DF42DEE0DC823071F0833030F4882356
:1008E000A1F0813009F085C04CC08330E1F0843044
:1008F00009F07FC07CC08091600190916101181661
:1009000019060CF076C0019709C0809160019091A2
:100910006101863091050CF06CC0019690936101E5
:100920008093600166C0E0916001F0916101EE0F7B
:10093000FF1FEE0FFF1FE05AFF4F80819181A281C0
:10094000B381209152013091530140915401509153
:100950005501820F931FA41FB51FE0914601F0912E
:100960004701EE0FFF1FEE0FFF1FE458FF4F2081DE
:10097000318142815381281739074A075B07CCF13F
:100980002DC0E0916001F0916101EE0FFF1FEE0FAD
:10099000FF1FE05AFF4F8091520190915301A091A7
:1009A0005401B09155012081318142815381821BD4
:1009B000930BA40BB50BE0914601F0914701EE0FAC
:1009C000FF1FEE0FFF1FEC56FF4F20813181428148
:1009D000538182179307A407B5075CF080935201F7
:1009E00090935301A0935401B093550102C011E0BC
:1009F00001C010E08FB580648FBD83EF91E0019757
:100A0000F1F700C000008FB58F7B8FBDD4DEA4DD71
:100A1000112309F45FCF1F910895CF92DF92EF92D7
:100A2000FF920F931F93DF93CF930F92CDB7DEB753
:100A3000AADB80E02DDB82ED90E090DB8FE996E889
:100A4000A1E081509040A040E1F700C00000E0909C
:100A50004601F09047011092470110924601CC24C4
:100A6000DD2480E415DBC114D10431F091E0C91616
:100A7000D10409F042C00CC082E191E06FDB0BDCD5
:100A800001E0843009F000E089837DDB898181C049
:100A900082EE90E063DBFFDB843009F079C0809167
:100AA000480190914901A0914A01B0914B01809376
:100AB000520190935301A0935401B093550107DF65
:100AC0008091520190915301A0915401B091550130
:100AD0008093480190934901A0934A01B0934B0140
:100AE000BB0F880B982FDC0180934C0180934D0144
:100AF00080934E0180934F013AC08601015010400F
:100B0000F801EE0FFF1FE65CFE4F8081918126DB2E
:100B1000C2DB8430E9F5A3E0000F111FAA95E1F7CD
:100B200004591E4FF80180819181A281B381809385
:100B3000520190935301A0935401B0935501C7DE25
:100B40008091520190915301A0915401B0915501AF
:100B50009C01AD01550F220B322FA901F8018083B2
:100B60009183A283B3832483258326832783E5DCB3
:100B700080E08EDA82E291E0F1DA8FE39DE0A3E09B
:100B800081509040A040E1F700C0000000E011C09B
:100B900000E0823021F0882341F0833021F4089472
:100BA000C108D10806C0813021F40894C11CD11CB1
:100BB00005C09FEFC9169FEFD90629F0A7E0CA1616
:100BC000D1042CF406C0E6E0CE2ED12C02C0CC24F9
:100BD000DD2480E05DDA82ED90E0C0DA8FB58064DC
:100BE0008FBDE3EFF1E03197F1F700C000008FB562
:100BF0008F7B8FBD002309F434CF8FB580648FBD08
:100C000087E893E10197F1F700C000008FB58F7B73
:100C10008FBDB9DAF0924701E0924601109252017D
:100C20001092530110925401109255010F90CF91E0
:100C3000DF911F910F91FF90EF90DF90CF9008957B
:100C40001F936CDCF894AEDB78948FB580648FBD15
:100C500083ED90E30197F1F700C000008FB58F7B23
:100C60008FBD83E090E090934701809346011092FE
:100C700052011092530110925401109255016CDCF4
:100C800080E406DA8AEF90E069DA80E001DA82E354
:100C900091E064DA00DB182F8FB580648FBD83EF9D
:100CA00091E00197F1F700C000008FB58F7B8FBDF9
:100CB000123051F42091460130914701121613066B
:100CC00094F4215030400BC0112369F42091460167
:100CD000309147012530310534F42F5F3F4F309379
:100CE00047012093460180E4D3D9E0914601F09179
:100CF0004701309741F48AED90E030DA80E0C8D9BE
:100D00008AE191E006C0EE0FFF1FE65CFE4F808196
:100D1000918124DA143041F4209146013091470149
:100D20002115310509F479DEE0914601F091470182
:100D3000309709F4AACF133031F01430E9F01130B4
:100D400009F0A3CF07C0EE0FFF1FEE0FFF1FE458FF
:100D5000FF4F06C0EE0FFF1FEE0FFF1FEC56FF4FB9
:100D600080819181A281B38180935201909353013C
:100D7000A0935401B0935501AADD87CF689401C0B8
:100D8000E8948F929F92CF93DF9305D0DF91CF911C
:100D90009F908F90089588249924F401E401B0E491
:100DA0001B2ED4019D158E049F04E007F10738F433
:100DB000FC014B01CA01B901AD019E011694220F3D
:100DC000331F441F551F661F771F881F991F881CDC
:100DD000991CEE1FFF1FCC1FDD1FAA1FBB1F8A140B
:100DE0009B04EC05FD05CE05DF05A007B10748F023
:100DF0008A189B08EC09FD09CE09DF09A00BB10B8D
:100E000021601A94E1F62EF49401AF01BE01CD01E8
:100E1000000C0895689401C0E894F92FF12B0AF0B2
:100E2000B0CFAA27BB27E6E1F7E0ADC0092E0594B5
:100E30001AF41BD0112392F4F0E80F26FFEFE09490
:100E4000F09400951095B094C094D094A194BF0AEA
:100E5000CF0ADF0AEF0AFF0A0F0B1F0B9CDF07FC0C
:100E600004D0CDB7DEB7ECE0AAC060957095809550
:100E7000909530954095509521953F4F4F4F5F4F3E
:100E80006F4F7F4F8F4F9F4F0895DF93CF931F93E7
:100E90000F939A9DF02D219FF00D8B9DF00D8A9D53
:100EA000E02DF10D039FF00D029FE00DF11D4E9D11
:100EB000E00DF11D5E9DF00D4F9DF00D7F936F9342
:100EC000BF92AF925F934F93D50130D08B01AC01AD
:100ED000D7012CD0EB01E80FF91FD6011FD02F91BD
:100EE0003F91D60123D0C60FD71FE81FF91FAF913E
:100EF000BF9114D02F913F9119D0C60FD71FE81F73
:100F0000F91FD60113D0E60FF71F9801BE01CF01DC
:100F100011240F911F91CF91DF91089507D0460FB3
:100F2000571FC81FD91F08F431960895A29FB0011A
:100F3000B39FC001A39F01D0B29F700D811D1124EA
:100F4000911D089597FB092E05260ED057FD04D05C
:100F50004BD00AD0001C38F450954095309521951F
:100F60003F4F4F4F5F4F0895F6F7909580957095DE
:100F700061957F4F8F4F9F4F08952F923F924F92D1
:100F80005F926F927F928F929F92AF92BF92CF9219
:100F9000DF92EF92FF920F931F93CF93DF93CDB722
:100FA000DEB7CA1BDB0B0FB6F894DEBF0FBECDBF9A
:100FB00009942A88398848885F846E847D848C846B
:100FC0009B84AA84B984C884DF80EE80FD800C8174
:100FD0001B81AA81B981CE0FD11D0FB6F894DEBF57
:100FE0000FBECDBFED010895A1E21A2EAA1BBB1BB7
:100FF000FD010DC0AA1FBB1FEE1FFF1FA217B307E5
:10100000E407F50720F0A21BB30BE40BF50B661FFA
:10101000771F881F991F1A9469F7609570958095BE
:1010200090959B01AC01BD01CF010895DC01CB017E
:10103000FC01E199FECF06C0FFBBEEBBE09A319602
:101040000DB20D9241505040B8F70895DC01A40F45
:10105000B51F4150504040F0CB01840F951F2E9199
:1010600005D041505040D8F70895262FE199FECF82
:101070009FBB8EBBE09A01970DB2021631F02DBBDB
:101080000FB6F894E29AE19A0FBE0895F894FFCF54
:1010900040420F00A086010010270000E803000076
:1010A000640000000A00000001000000FFFF0F00C4
:1010B00040420F0040420F0040420F0040420F00EC
:1010C00040420F000000000000000000000000008F
:1010D0000000000000000000000000000700030006
:1010E00001000200030001001D4C6F92004C6F9242
:1010F000B81D2044432D43616C204E616E6F205615
:101100002E32436F72726563743A2043616C696278
:10111000723F202020305620202020203130306D9A
:10112000562020202031562020203130562F3130BB
:101130006D412020313030562020202020314120A8
:101140002020202045786974202020202020202085
:1011500020202020204F6B2120205374617274695D
:101160006E673C53656C6563743EDA00EA00F2001A
:06117000FA0002010A0171
:00000001FF
